S00D000070705F476E6F6D5F31335F
S1130000A1C01895189518951895189518951895D0
S1130010189518950150104098018901232BD1F7A8
S1130020089512E813BF06BF00E21EE4F3DF00E008
S113003003BF08958ED0B99ABC9A02EE06B903E0C4
S113004007B900E21EE4E6DF02E50FBD00E808B9E7
S1130050C49A00E2E6DF00E4E4DF00E8E2DF00E166
S113006017E2D8DF00E2DDDFC49800E003BF08EE4A
S11300701DEFD0DF4424552490E06624772480E0EB
S11300800CC035B120E004B110E0202B312B620EFE
S1130090731E04E110E0BEDF8395803490F399234E
S11300A011F4D30197E09D0126193709213000E8A6
S11300B0300710F020E030E0223400E03007C8F0D0
S11300C09394092D902E053060F0992444245524EE
S11300D0C49A3695279536952795209526BF01E82D
S11300E003BFAA248394082D802E002369F490E092
S11300F00BC0C49800E003BF88249924A3940A2D5C
S1130100A02E002309F490E001E0400E00E0501E10
S11301108201280101322EE4120708F4AECF4424F0
S1130120552480E0833008F0A8CFC49A00E779DF33
S1130130C49800E41CE96EDF90E08395F3CF0000DF
S11301408895FECF0FE90DBFC0E80FD073DFF7DF4E
S1130150F6CFAA929A928A927A926A925A924A9282
S1110160BA93AA939A938A93089501E008959E
S9030000FC
